:100000000C9434000C9451000C9451000C94510049
:100010000C9451000C9451000C9451000C9451001C
:100020000C9451000C9451000C9451000C9451000C
:100030000C9451000C9451000C9451000C945100FC
:100040000C9451000C9451000C9451000C945100EC
:100050000C9451000C9451000C9451000C945100DC
:100060000C9451000C94510011241FBECFEFD4E02A
:10007000DEBFCDBF11E0A0E0B1E0E8E0F1E002C0FA
:1000800005900D92A030B107D9F711E0A0E0B1E0E2
:1000900001C01D92A030B107E1F70E945D000C94F1
:1000A00082000C94000020EE31E004C0F901319789
:1000B000F1F701970097D1F708951DBA10926800E3
:1000C00010926C0080916C0080936B008FE38AB972
:1000D00084E087B96FE054E020EE31E040E36BB993
:1000E00058B986E990E0F9013197F1F70197D9F70E
:1000F0004BB918B886E990E0F9013197F1F701970B
:08010000D9F7EDCFF894FFCF11
:00000001FF
